:020000040800F2
:1000000000020020BD04000849040008590400084B
:100010006904000879040008890400080000000051
:100020000000000000000000000000000D040008B7
:100030009904000800000000F1030008A90400086A
:100040008901000889010008890100088901000868
:100050008901000889010008890C0008890C000842
:10006000890C0008890C0008890C00088901000827
:100070008901000889010008890100088901000838
:100080008901000889010008890100088901000828
:10009000890100088901000889010008890C00080D
:1000A0008901000889010008890100088901000808
:1000B0002D11000889010008890100088901000844
:1000C00089010008890100088901000889010008E8
:1000D0008901000889010008150B00081B0B0008A6
:1000E000890C0008890100088901000889010008BD
:1000F00089010008890100088901000889010008B8
:1001000089010008890100083311000889010008ED
:100110008901000889010008890100088901000897
:100120008901000889010008890100088901000887
:100130008901000889010008890100088901000877
:100140008901000889010008890100088901000867
:100150008901000889010008890100088901000857
:100160008901000889010008890100088901000847
:1001700089010008890100088901000800000000C9
:10018000000000008901000800F08EB900F0F8B905
:100190007047000070B50C46064600F045F9094B63
:1001A000094A1D682919914202D8084A914204D28D
:1001B0000C2333604FF0FF3500E0196000F03CF98C
:1001C000284670BD0002002000000220880B00209D
:1001D0001946104600F0E0B91946104600F0E4B99F
:1001E000132303604FF0FF307047132303604FF079
:1001F000FF307047132303604FF0FF307047022930
:100200004FF0000303608CBF002001207047000006
:10021000114B70B500241C60104B114D18682E68EE
:1002200000F09CF80F4B53F820301B68A3F1080234
:1002300096420FD026B13179092904BF0A213171C4
:10024000092103F8041C33F9021C074B2A601980AA
:10025000012070BD204670BD8C020020600300208C
:10026000940200209C02002090020020082930B552
:10027000037919D9082B32D842791A4B53F82250F6
:1002800000F108042DB12D68856053F822502C60D0
:1002900000E0846043F82240134C4279012303FAC2
:1002A00002F22368134319E0082B18D945790D4B46
:1002B00053F825203AB11468A2420BBF00222468EB
:1002C00043F825201460427953F822303BB9064C9C
:1002D000012303FA02F2236823EA02032360017177
:1002E00030BD00BF9C0200206003002008B50A4B0F
:1002F0001B681A79082A02D95B7983420AD900F06F
:100300009EF818B1054B01221A6008BDBDE80840EF
:1003100000F066B808BD00BF940200208C020020E7
:1003200008B500F081F8094B094A1B88094D1BB23A
:10033000002442F82340084A286813682146013BFC
:100340001360FFF793FF2C6000F046F89002002046
:10035000DC02002094020020980200200023C20743
:1003600002D440080133FAE718467047134423F0DB
:10037000030310B54FF077321C1F43F8042C6207BB
:1003800042BF4FF0883243F8082CA3F108044FF025
:10039000807304E909000F4B44F80C3C002344F837
:1003A000103C032344F8143C2246022344F8183C32
:1003B000012344F81C3C42F8201D0B2342F8043D65
:1003C000013B032BFAD120466FF0020340F8443D75
:1003D00010BD00BF2103000800F02AF801DFFEE78E
:1003E000024A536843F080535360704700ED00E0C9
:1003F000EFF3098020E9F00F40F804ED02490968A5
:10040000086000F003F8000094020020FFF700FFEE
:1004100004480068016801C9B1E8F00F81F3098858
:100420000047000094020020EFF3108072B670477E
:1004300062B6EFF31080704780F310887047EFF3D7
:100440000580C0B27047000008B50249042000F0E2
:10045000D5F800BF3829000808B50249052000F08A
:10046000CDF800BF4429000808B50249062000F075
:10047000C5F800BF5729000808B50249072000F059
:10048000BDF800BF6A29000808B50249082000F03D
:10049000B5F800BF7C29000808B50249092000F022
:1004A000ADF800BF9029000808B502490A2000F005
:1004B000A5F800BFA22900087047704708B5FFF7EC
:1004C000FBFF0E4A0E4B0F498B4204D252F8040F29
:1004D00043F8040BF8E70C4B0C4A0021934202D27C
:1004E00043F8041BFAE7FFF7E8FF00F067F800F0B5
:1004F00023FEBDE8084000F0A9B800BFD42E0008D4
:10050000000200208C0200208C020020880B0020BA
:1005100010B568B1012815D1174A136823F00303F9
:100520001360136843F4007343F0010313601BE08E
:10053000114B1A6842F00E021A605A6842F4807237
:100540005A6011E00D4A136923F00403136100247B
:10055000FFF76AFFBFF34F8F30BFFFF76DFF54B156
:10056000BDE8104000F08EB9044A136943F004035B
:1005700013610124ECE710BD0070004000ED00E0C5
:10058000034B044A4FF4E131002000F04DBA00BFA4
:1005900004020020FF0700080A460146014800F057
:1005A00039B900BF0402002010B50A460C460146C6
:1005B000002000F095FA204610BD000008B501218A
:1005C000094800F0F5FA0121084800F0F1FA01218C
:1005D000074800F0EDFA0121064800F0E9FABDE80D
:1005E000084000F003B900BF0D0C02400C0C0240A3
:1005F0000E0C02400F0C02407047000008B5084B7B
:100600001A683AB9012207481A6000F021FE06482C
:1006100000F01EFEFFF708FFFFF7EEFF00F0D4F832
:10062000A4030020B0290008CC29000808B500F078
:1006300045FC034800F00CFE00F086FB002008BDDE
:10064000DF29000808B500F0FFF8FCE71FB5FFF749
:10065000EBFE0E4B0E481B68029300240D4B0093DB
:100660000F220C234FF48071019400F045F80A4BDF
:100670000A481B6802930A4B009307220C234FF48D
:10068000C061019400F038F8FFF7A6FE18020020C0
:10069000A8030020450600081C020020A804002032
:1006A0002D06000808B5FFF7BFFE094B1B681A7935
:1006B000082A07D95A79074B53F8221011B1096853
:1006C00043F82210FFF7B8FEBDE80840FFF788BEE8
:1006D000940200209C02002030B54C7901F1080200
:1006E00003682BB113F8035CAC4201D31846F7E75B
:1006F0008B60026030BD00000F2A2DE9F84F804664
:1007000091469A4620D810F003031CBFC3F104039E
:10071000C91AA1F1240118BF984421F00307FFF77B
:1007200083FE274A08EB07048346012352F823601F
:100730001DB26EB10133212BF8D15846FFF77CFE74
:100740006FF08A00BDE8F88F6FF01500BDE8F88FF4
:100750001B4A0B9942F823400A98E5803B464246E3
:10076000FFF704FE174A20604FF0FF33E361136880
:1007700084F8059001331AF0010F2671A660E66037
:1007800026616661A6612662136004D001212046BD
:10079000FFF76CFD0DE00A212046FFF767FD1AF018
:1007A000040F06D15846FFF747FE4846FFF79EFD67
:1007B00002E05846FFF740FE2846BDE8F88F00BF2C
:1007C000DC02002098020020BFF34F8F0549064B42
:1007D000CA6802F4E0621343CB60BFF34F8F00BFDF
:1007E000FDE700BF00ED00E00400FA0508B500F0E9
:1007F000BDFB00F047F8BDE8084000F01CB838B574
:100800000446043000F07DFA0546204600F088FBDF
:10081000284638BDF8B504460E461746051D3A462B
:100820003146284600F058FA20B90121204600F050
:1008300047FBF4E7F8BD08B5002000F095F901206A
:10084000BDE8084000F090B9F8B50D4B1E68C6F33E
:1008500007221D4622B9F4B2003418BF012400E07B
:100860000224FFF7E1FD2B689E42074602D1204695
:10087000FFF74EFE3846BDE8F840FFF7DDBD00BF8C
:100880002002002038B5FFF7CFFD1B4C0023E360AA
:10089000054600F037F84FF41443A360A268164BE6
:1008A00012F00C0FFAD1154A40F205711160812245
:1008B0001A601A6842F480321A601A6812F4003F13
:1008C0000D4AFAD00E4B5360136843F080731360E7
:1008D0001168094B8901FBD59A6842F002029A60BF
:1008E0009A6802F00C02082AFAD100F017F828469C
:1008F000BDE83840FFF7A0BD00380240003C024090
:10090000042A4007044B1A6842F001021A601A6870
:100910009207FCD5704700BF00380240044B9A682C
:1009200012F00C0F1EBF1A6822F001021A60704705
:1009300000380240034B044A00280CBF10461846FA
:10094000704700BF00BD010580DE800204281CD86E
:10095000DFE800F003080D1217000D4B1A6C11436D
:10096000196412E00A4A536C194351640DE0084AB5
:10097000136B1943116308E0054A536B1943516324
:1009800003E0034A936B19439163BFF34F8F7047A2
:1009900000380240042821D8DFE800F003090F15D1
:1009A0001B000F4A136C23EA0101116470470C4AC3
:1009B000536C23EA010151647047094A136B23EA1F
:1009C000010111637047064A536B23EA0101516329
:1009D0007047034A936B23EA01019163704700BF9C
:1009E0000038024038B514230C4A4343D4582568D4
:1009F000AA0608D50A4B616803EBC002C9B253F8D6
:100A00003030506898472B0748BF6368054B1B6818
:100A10001BB1BDE83840FFF745BE38BD382A000895
:100A2000A80A00208C0200202DE9F843DFF8AC90E2
:100A3000142404FB00941746264AE66842F83070F6
:100A400002EBC0028046536030460D46012100F0A3
:100A5000AFF8304600F00EF93046617C00F0E2F865
:100A60004E464FB1D4F808900021484600F0A0F857
:100A7000217C484600F0D6F8142303FB08F406EB6B
:100A8000040898F81290D8F804104846FFF75EFF63
:100A900034590023E360484623616361FFF74AFF4E
:100AA000B0FBF5F080B2A06077B198F81330012167
:100AB0005AB203F01F0301FA03F35209064941F841
:100AC000223042F22C0301E042F20803E3600020EE
:100AD000BDE8F883A80A002000E100E0382A0008F9
:100AE00030B50B4C14230A4403FB0043914207D05A
:100AF0001C6825682D06FCD511F8015B6560F5E7DB
:100B000014235843024B1A5813685B06FCD530BDBA
:100B1000382A00080020FFF765BF0120FFF762BFF9
:100B2000F8B5104C04EB401401216768384600F01A
:100B30003FF8A6680021304600F03AF8E568012148
:100B4000284600F035F8247D3846214600F06AF842
:100B50002146304600F066F821462846BDE8F840B8
:100B600000F060B8602A00080F4B2DE9F041002525
:100B70000446DFF8388043F820506401FFF7D0FFC7
:100B800008EB04031E7F9F6930463946FFF7DEFEFF
:100B900058F8043039461D603046DD615D60BDE8BF
:100BA000F041FFF7F7BE00BFB80A0020602A000836
:100BB000F8B50D460126C0F3832120F00F0400F0A4
:100BC0000F0706FA01F10220FFF7C0FE07FA06F050
:100BD0000323216883406FEA030C01EA0C012160C2
:100BE000216805F0030E0EFA00FE4EEA01012160B5
:100BF000E2680CEA0202E260E168C5F38102824029
:100C00000A43E2606268BE4022EA060666606268E5
:100C1000C5F30015BD4015436560A2681343A3608A
:100C20000020F8BD20F00F0300F00F02F0B51E68A1
:100C300057000325BD4026EA05051D601D680224F6
:100C4000072A04FA07F444EA050494BF00220122AB
:100C50001C6003EB820300F007001C6A80000F2277
:100C6000824024EA02021A621A6A814041EA0200C2
:100C70001862F0BD20F00F02012300F00F0003FA0C
:100C800000F0906170470000104B2DE9F0415E6963
:100C90001A680F4F164000244FF001081D4608FA4D
:100CA00004F31E4206D06B6107EBC40357F83420EF
:100CB000586890470134102CF1D1064B1B681BB1CA
:100CC000BDE8F041FFF7EEBCBDE8F081003C01401B
:100CD000C00A00208C02002070B513467BB18568E5
:100CE000C468A5420BD084680668651C85604568A9
:100CF000013D2C40013B345D01F8014BEEE7D01A79
:100D000070BDC368426830B584681B1B934208D02D
:100D1000C3680468013A5D1C1340C560E1540020BB
:100D200030BD4FF0FF3030BD044B1A68044B43F820
:100D30002120044A1368013313607047440B0020DC
:100D4000480B0020400B00202DE9F74F4748484E44
:100D500000F008FB474800F005FB0221464800F080
:100D600077FA0024A146A24621464448444F00F0A9
:100D70006FFA444A0023C2F800A09046C7F800A0CA
:100D800046F823A001330A2BFAD13F493F4A0023FA
:100D9000204600F07DF90028214604DA3C4800F0A6
:100DA00057FA002553E03B4800F052FA204600F085
:100DB000B3F92146384800F04BFA00256B1C41F28C
:100DC000883202FB03FB5A462946204601930095D0
:100DD00000F0F0F80028019B05DA6DB921462F4894
:100DE00000F036FA33E01D46009A2D485B46214656
:100DF00000F02EFA0A2DE1D121462A4800F028FA07
:100E0000204600F03BF9D8F800300133C8F8003034
:100E10003B689D42F7D100253B689D4216DA144B92
:100E2000214853F825302A46214600F011FA15B919
:100E300031681E4806E06B1E56F8251056F8233020
:100E40001B48C91A00F004FA0135E5E70125013411
:100E5000022CA94488D1B9F1020F0CBF15481648DD
:100E600000F080FA002003B0BDE8F08FA02A00084F
:100E7000480B0020BD2A0008BE2C0008D42C000816
:100E8000400B0020440B002040420F00290D0008B9
:100E9000E82C0008172D00083C2D00086F2D0008D5
:100EA0004F2D0008952D0008A92D0008D42D00080D
:100EB000E22D0008F02D0008002E00087047000009
:100EC00070B505460C46FFF7AFFA2B6806462BB9FE
:100ED0004FF0FF332B60FFF7AFFA18E0CCB10F4BA8
:100EE0001C6802212046FFF7C1F92B68013305D1A8
:100EF00004F108032B600023A36003E02146284689
:100F0000FFF7EAFB3046FFF797FAFFF769FA01208F
:100F100070BDFFF791FA204670BD00BF940200201B
:100F200070B50446FFF780FA256806461DB16B1CB4
:100F300005D100232360BDE87040FFF77DBA284645
:100F40000A2150F808392360FFF790F9236813B994
:100F50004FF0FF33236015F8034C3046FFF76CFA6F
:100F60002046BDE87040FFF7C1B900000F4BD3F831
:100F7000882042F47002C3F888200D4A9A6010223B
:100F800083F822200021DA7701F1604000F561400A
:100F90000131522980F80023F6D11A6942F010027B
:100FA0001A615A6942F400725A61704700ED00E01C
:100FB0000000000870B504460D46164600F056F8CD
:100FC000294682192046BDE8704000F02FB8000085
:100FD0002DE9F843124ADFF8508003010746D5583F
:100FE0002E69EB6800241E4008EBC0090223A340D1
:100FF0001E4209D0EA68D9F8040022EA0303EB6034
:10100000214658F8373098470134042CEED1054B6F
:101010001B681BB1BDE8F843FFF744BBBDE8F8838C
:10102000102E00088C020020700B0020032910B540
:1010300016D80D4B00011C181B586068024001F1C6
:101040000C0003EB800042601869022202FA01F1F1
:1010500020EA01021A61DA681143D960002010BD4C
:101060004FF0FF3010BD00BF102E00080001024BF2
:101070001B58586A704700BF102E0008034B000130
:101080001A58136843F0010313607047102E0008CC
:1010900001282DE9F8430546884630D81A4E1B49E9
:1010A0000401371941F8302097F80C9001EBC0018A
:1010B00048464B60B968FFF749FC36597B68002405
:1010C000346048467460F362FFF734FC104B7A7B5F
:1010D00013F809305843B0FBF8F3013BB36251B247
:1010E000012302F01F02736149099340094A28460F
:1010F00042F82130FFF7C2FF2046BDE8F8834FF0E9
:10110000FF30BDE8F88300BF102E0008700B0020F0
:10111000302E000800E100E0034B00011A5813686C
:1011200023F0010313607047102E00080020FFF722
:101130004FBF0120FFF74CBF70B50F4E0F4D761B10
:10114000B61018BF002405D0013455F8043B984769
:10115000A642F9D10A4E0B4D761BFFF717F8B610D1
:1011600018BF002406D0013455F8043B9847A64226
:10117000F9D170BD70BD00BFD82E0008D82E000870
:10118000D82E0008D82E000870B4840746D0541E0C
:10119000002A41D0CDB2034602E0621EE4B31446F9
:1011A00003F8015B9A07F8D1032C2ED9CDB245EA9A
:1011B00005250F2C45EA054519D903F110022646ED
:1011C000103E0F2E42F8105C42F80C5C42F8085CAE
:1011D00042F8045C02F11002F2D8A4F1100222F0ED
:1011E0000F0204F00F041032032C13440DD91E46D5
:1011F0002246043A032A46F8045BFAD8221F22F05A
:1012000003020432134404F003042CB1C9B21C4499
:1012100003F8011BA342FBD170BC70471446034680
:10122000C2E700BF0EB410B5044683B018B183699D
:101230000BB900F04DFB06A803460190059AA16882
:10124000204600F007FD03B0BDE8104003B0704732
:101250000FB410B50A4B1C6882B024B1A36913B94E
:10126000204600F035FB05A803460190049AA168CA
:10127000204600F0EFFC02B0BDE8104004B070471B
:10128000240200202DE9F0410E46804600283ED081
:101290008369002B39D084682F4B9C4243D02F4B5D
:1012A0009C4256D02E4B9C4208BFD8F80C40A389D4
:1012B0001B073DD52369002B3AD0013EA36816F8E1
:1012C000015F013BA360B5B1002B04DB23685A1C0E
:1012D00022601D70F2E7A769BB42224629464046BC
:1012E00001DB0A2DF2D100F045F80130E6D14FF0D4
:1012F000FF30BDE8F081002B21DB23680A22591C56
:1013000021601A701046BDE8F08100F0E1FAD8F8CB
:101310001830D8F80840002BBED1404600F0D8FA6B
:101320000D4B9C42BBD1D8F80440A3891B07C1D404
:101330002146404600F080F80028BED0D7E722467C
:1013400040460A2100F016F80130D0D00A20BDE84E
:10135000F081D8F80840AAE77C2E00085C2E00082F
:101360003C2E0008024B01461868FFF78BBF00BFF8
:1013700024020020F8B50E461446054610B18369D4
:10138000002B41D0254B9C4243D0254B9C4242D060
:10139000244B9C4208BFEC68A389A269A2601A078B
:1013A00021D52369FBB122686169D31A8B42F7B258
:1013B00021DA0133A168501C0139A1602060167048
:1013C00062699A4206D0A389DB0701D50A2F01D0B2
:1013D0003846F8BD2146284600F040F90028F7D0ED
:1013E0004FF0FF37F4E72146284600F025F80028A3
:1013F000F6D12369D7E72146284600F02FF90028C7
:10140000EED122680123D5E700F062FA034B9C423B
:10141000BBD16C68C0E7AC68BEE700BF7C2E00089B
:101420005C2E00083C2E0008024B0A460146186854
:10143000FFF7A0BF24020020384B70B51D68064698
:101440000C4615B1AB69002B42D0354B9C4245D0C0
:10145000344B9C4258D0344B9C4208BFEC68B4F9E2
:101460000C2093B219070CD52069A8B113F0010222
:101470001ED0636900225B42A361A260F0B100202C
:1014800070BDDD0642D558072AD4206942F0080312
:10149000A3819BB20028E9D103F42072B2F5007F4A
:1014A000E4D03046214600F0B1FAA3892069DDE797
:1014B000990758BF6269A2600028E0D1B4F90C30E6
:1014C0001A06DDD543F04003A3814FF0FF3070BD15
:1014D000284600F0FDF9124B9C42B9D16C68BEE77A
:1014E000616B51B104F14403994204D0304600F0DD
:1014F000D1FAB4F90C2000236363002320696360F0
:1015000022F024022060C1E7AC68A8E742F0400264
:10151000092333604FF0FF30A28170BD2402002008
:101520007C2E00085C2E00083C2E00088B891A07D0
:101530002DE9F0410D46804635D44A68002A6BDD1E
:10154000EC6A002C47D003F48052002192B2D8F804
:101550000060C8F80010002A62D06A6D5F0705D5E8
:1015600069686B6B521A0BB12B6CD21A0023296A73
:101570004046A047441C39D0AB892A692A60DB0465
:101580004FF000026A6045D4696BC8F8006011B37F
:1015900005F14403994202D0404600F07BFA002056
:1015A0006863BDE8F0810E69AEB10C680E60980703
:1015B0000CBF4B690023A41B8B600AE02346324614
:1015C000AF6A296A4046B8470028A4EB00040644E5
:1015D00004DD002CF2DC0020BDE8F081AB8943F093
:1015E0004003AB814FF0FF30BDE8F081D8F8002018
:1015F0001D2AF3D8184BD34003F0010383F00101F7
:10160000002BEBD0AB892C696960D9042C60BBD569
:10161000002AB9D16865B7E70A6C002A90DCDAE7DE
:101620000123296A4046A047431C024602D0AB89E9
:10163000EC6A93E7D8F80030002BF8D01D2B01D0CE
:10164000162B02D1C8F80060C5E7AB8943F0400310
:10165000AB81BDE8F08100BF010040200B6933B3CE
:1016600010B5044682B008B18369ABB1114B994201
:1016700019D0114B994218D0104B994208BFE1681C
:10168000B1F90C3013B9002002B010BD204602B0F1
:10169000BDE81040FFF74ABF019100F019F9019928
:1016A000044B9942E5D16168EAE7A168E8E70020C8
:1016B000704700BF7C2E00085C2E00083C2E0008FE
:1016C00020B1054B01461868FFF7C8BF034B04491A
:1016D000186800F043B900BF24020020342E00082F
:1016E0005D16000800207047014900F037B900BFBF
:1016F0005D1600080020704770B568234D1E03FB7F
:1017000005F50E4605F1740100F00AFA044640B1F1
:1017100000210C30666005F168022160A060FFF7CF
:1017200033FD204670BD00BF1F4B70B51D68AB690F
:10173000064613B9284600F039F848356B68AC689E
:10174000013B05D521E0013B5A1C04F168041CD083
:10175000B4F90C20002AF6D1002501234FF6FF72C0
:10176000E281A38165662560A5606560256165618C
:10177000A5612946082204F15C00FFF705FD6563B9
:10178000A563A564E564204670BD2B680BB11D46BA
:10179000D4E704213046FFF7AFFF286008B10546C3
:1017A000CCE70C23336070BD342E00083D4B3E491E
:1017B0001A682DE9F04F90424FF000038364C36430
:1017C000036508BF012383B008BF836181620746B8
:1017D000FFF7AAFF78603846FFF7A6FFB8603846E3
:1017E000FFF7A2FF7D68F86000240423AB812C6022
:1017F0006C60AC606C66EC812C616C61AC61214604
:1018000005F15C000822FFF7BFFCBE68DFF89CB062
:10181000DFF89CA0DFF89C90DFF89C80C5F824B02E
:1018200001230922C5F828A0C5F82C90C5F83080FE
:101830002D622146F381B28134607460B4607466B5
:1018400034617461B46106F15C0008220193FFF712
:101850009BFCFD68366212200222C6F824B0C6F84E
:1018600028A0C6F82C90C6F830802146A881EA81CD
:101870002C606C60AC606C662C616C61AC6105F1D5
:101880005C000822FFF780FC019B2D62C5F824B0A4
:10189000C5F828A0C5F82C90C5F83080BB6103B00E
:1018A000BDE8F08F342E0008E9160008AD220008CC
:1018B000D52200081123000831230008024B0349F8
:1018C000186800F04BB800BF342E00085D16000801
:1018D000836903B96AE77047704700BF704700BF6C
:1018E000704700BF704700BF024B0349186800F003
:1018F0000FB800BF24020020F5160008024B034970
:10190000186800F005B800BF24020020E5160008A2
:101910002DE9F04110F148071BD0884600267D686C
:10192000BC68013D0FD4A389012B05F1FF3506D911
:10193000B4F90E300133204601D0C04706436B1C7A
:1019400004F16804EFD13F68002FE8D13046BDE8CC
:10195000F0813E463046BDE8F08100BF2DE9F843F6
:1019600010F148071FD0884606464FF000097D68F1
:10197000BC68013D11D4A389012B05F1FF3508D9BD
:10198000B4F90E3001332146304602D0C04749EA4F
:1019900000096B1C04F16804EDD13F68002FE6D10B
:1019A0004846BDE8F883B9464846BDE8F88300BF1D
:1019B00070B50C46B1F90E10002990B015461E46C0
:1019C00013DB01AAFEF716FC00280EDB029A02F4D4
:1019D0007042A2F50052B2FA82F252094FF48063CB
:1019E000002032602B6010B070BDA38900221B065E
:1019F000326004D5402300202B6010B070BD4FF43E
:101A0000806300202B6010B070BD00BF8A899207F0
:101A10000B4606D501F1470201211A601A6159618E
:101A20007047F0B583B001AB6A460C460546FFF738
:101A3000BFFF00990646284600F072F8B4F90C3052
:101A4000D0B1019A124F0099AF6243F08003A38195
:101A50002060206161611AB93343A38103B0F0BDF6
:101A60002846B4F90E10FEF7CAFBB4F90C30002872
:101A7000F2D043F00103EFE79A05EFD404F14702F7
:101A800043F002030121A381226022616161E5E745
:101A9000E916000830B481B151F8043C0439002B38
:101AA000B8BFC9181D4B1A682AB18A420AD90868FA
:101AB0000C18A24225D04A60196030BC70478B4296
:101AC00003D81A465368002BF9D1146815198D42B2
:101AD0000CD007D808680C189C4218D04B6030BC5A
:101AE000516070470C23036030BC704709680C4498
:101AF000111999421460E0D10ACB0C445360146070
:101B0000DBE7146852684A6020440860D4E71C6828
:101B10005B684B60204408605160CEE7800B00207A
:101B200070B5CD1C25F0030508350C2D38BF0C25EC
:101B3000002D06463BDBA94239D827490A6852B135
:101B400013685B1B04D436E023685B1B1AD522465E
:101B50005468002CF8D149681F4C002936D029461A
:101B60003046FEF717FB431C21D0C41C24F00304AD
:101B7000A04205D0211A3046FEF70CFB013016D0EA
:101B8000256004E00B2B0DD923601C44256004F173
:101B90000B0020F00700231DC31A02D05A42E25066
:101BA00070BD70BD94420ED063685360EFE70C23A4
:101BB0003360002070BD0B2B03D8536814460B60B4
:101BC000E5E71446E0E713461446F8E73046FEF72B
:101BD000E1FA6060C3E700BF800B00209368013B1F
:101BE000002B10B4936007DBCCB21368581C106054
:101BF0001970204610BC70479469A34202DBCCB236
:101C00000A2CF2D110BCFFF7B5BB00BF93B1F8B5F9
:101C100014460F460646D51801E0AC4208D03A46B5
:101C200014F8011B3046FFF7D9FF431CF5D1F8BD6E
:101C30000020F8BD00207047936810B5144613B912
:101C40005360184610BD00F077FB0023A36063606B
:101C500010BD00BF2DE9F04F9DB088461446039398
:101C6000814618B18369002B00F00B818B4B98459E
:101C700000F00D818A4B984500F00C81894B984506
:101C800008BFD9F80C80B8F80C301D0740F1EF8080
:101C9000D8F81030002B00F0EA8030238DF82A307D
:101CA0002378814DDFF804A20021202209918DF8CC
:101CB0002920002B00F08580252B264603D117E034
:101CC000252B00F0868016F8013F002BF8D1B6EBEB
:101CD000040B76D022465B4641464846FFF796FF06
:101CE00001306ED0099B32785B440993002A68D09A
:101CF00000234FF0FF31721C0493079306938DF875
:101D000053301A930591012604E0049906FA03F36F
:101D10000B430493144664482178052200F090FC9C
:101D2000621C431B0028F0D1049BD80644BF20222C
:101D30008DF853201907217844BF2B228DF85320AA
:101D40002A2968D0A1F13002092A0BD8079B14F880
:101D5000011F03EB830302EB4303A1F13002092AC5
:101D6000F5D907932E293FD00322504800F068FC94
:101D700048B10499CAEB0000402202FA00F041EA9F
:101D8000000301340493217849488DF82810062275
:101D9000013400F055FC00285FD0464BEBB103AB9B
:101DA00000934246444B04A94846AFF300800746DF
:101DB0007A1C06D0099B3B4409932378002B7FF4BF
:101DC0007BAFB8F80C305B0658D409981DB0BDE85D
:101DD000F08FB6EB040B8BD07CE7039B073323F02B
:101DE000070308330393E5E761782A291DD0A1F1A1
:101DF00030020023092A04F101040593B4D814F831
:101E0000011F03EB830302EB4303A1F13002092A14
:101E1000F5D90593A8E7039A1168043200290392C3
:101E200015DB0791617801349CE7039B1A680592E2
:101E3000002A03F104030393B8BF4FF0FF3204F10B
:101E40000203AEBFA178A17805921C468CE74942F7
:101E500043F0020307910493E4E703AB0093424687
:101E6000154B04A9484600F0CDF80746A0E74146C7
:101E70004846FFF7E1FA00283FF40FAF4FF0FF307C
:101E8000A4E7FFF725FD054B98457FF4F3AED9F89D
:101E90000480F8E6D9F80880F5E600BF7C2E00083B
:101EA0005C2E00083C2E00089C2E0008A42E000882
:101EB000A82E0008000000000D1C000810B4044CFF
:101EC00013460A460146206810BCFFF7C3BE00BF98
:101ED000240200202DE9F0470C4691460969A268CA
:101EE000DDF820808A42B8BF0A46C9F8002094F87D
:101EF000431006461F4611B10132C9F8002023687D
:101F000099065DD5D9F800200232C9F8002023686F
:101F100013F0060F19461DD1E1688A1A002AD8BFAE
:101F2000194617DD04F1190A002505E0E368D9F820
:101F300000209B1AAB420CDD012352463946304645
:101F4000C047013005F10105F0D14FF0FF30BDE889
:101F5000F087216894F84330003318BF01238A06C4
:101F60000AD5E1185A1C302081F84300224494F825
:101F7000451082F84310023304F1430239463046DB
:101F8000C0470130E1D0236803F00603042B29D0B9
:101F9000A36822699342C8BF4FF000092FDD9B1A46
:101FA00099441A34002501E04D4528D001232246EA
:101FB00039463046C047013005F10105F4D1C4E788
:101FC00013F0060F08D1E168D9F800208A1A002A18
:101FD000D8BF1946A6DCBDE794F84330003318BFDC
:101FE0000123C9E7D9F80000E168A3682269091A4A
:101FF000934221EAE179D2DCB9F1000FD1D100207E
:10200000BDE8F0872DE9F0430C46097E85B06E29C6
:10201000064617460C98984604F1430C5AD01AD835
:10202000632900F0128100F2D68000295CD0582983
:1020300040F0F58084F8451022680368DFF864E218
:10204000150603F104011ED4550653BF1B68016039
:102050001B88016019E0732900F0CF807ED86F29BA
:1020600000F0E480702940F0DA80226842F020021B
:102070002260782384F845300368DFF82CE21506E7
:1020800003F10401E0D51B680160D00744BF42F0B2
:1020900020022260002B40F09080226822F0200273
:1020A00022601021002284F843206068A06000288C
:1020B000C0F28880226822F004022260002B62D1E4
:1020C000002840F08180654608296AD0C5EB0C03E2
:1020D00023610CE023681A0640F1D5800368626929
:1020E000191D01601B681A60002365462361CDF845
:1020F00000803B4603AA21463046FFF7EBFE013045
:1021000021D02A46236939463046C04701301AD0CB
:102110002368039813F0020FE36819D01A1A002AF3
:1021200016DD04F11909002504E0E36803981A1A82
:10213000AA420DDD01234A4639463046C0470130E8
:1021400005F10105F1D14FF0FF3005B0BDE8F08396
:102150009842B8BF184605B0BDE8F083752965D030
:1021600078295CD1226884E76168A1602D2000296C
:10217000C3F1000384F8430021DB22F00402DFF8FE
:1021800024E122600A216546B3FBF1F201FB123023
:1021900013461EF8002005F8012D002BF4D1082964
:1021A00094D12368D90791D5626823699A428DDC5E
:1021B000302305F8013C013D88E7102172E7DFF884
:1021C000E4E00A21002BDED19EF8003084F8423092
:1021D00004F1420578E7642901D069291FD12268FA
:1021E0000368150603F104013AD51B680160002B52
:1021F000BADBDFF8B0E00A2157E703686268191D0F
:1022000001601D680021284600F01AFA002846D017
:10221000401B60602061002384F8433067E701239E
:1022200084F84210236104F14205F4E723681A069A
:102230001ED503681A1D1B680260227EDFF864E069
:102240006F2A14BF0A2108212CE703681A68191D98
:102250000123016004F1420584F842202361DAE79A
:10226000550653BF1B680160B3F900300160BEE73B
:1022700013F0400F036803F1040215BF02601B68EE
:102280001B880260D9E713F0400F0368626903F10D
:10229000040101601B6814BF1A801A6024E760689B
:1022A000B8E700BFB02E0008C42E000810B50C46D9
:1022B000B1F90E10FDF78CFF002803DB636D0344BA
:1022C000636510BDA38923F48053A38110BD00BFB3
:1022D000002070472DE9F0411646B1F90C201F4649
:1022E000D3050C46054607D500220223B1F90E108E
:1022F000FDF77BFFB4F90C20B4F90E1022F48052E4
:10230000A2813B4632462846BDE8F041FDF764BF56
:1023100010B50C46B1F90E10FDF767FFA389421CFA
:102320000EBF23F4805343F480536065A38110BD36
:10233000B1F90E10FDF754BF9368002B76D02DE94C
:10234000F04F8B8985B00C4619070190164629D5A8
:1023500022693AB303F002081FFA88F035680028B2
:102360002FD04FF00009B44FC846B246B845434697
:102370004A4628BF3B460198B8F1000F50D0216A69
:10238000A66AB047002871DDDAF808301B1A8144CC
:10239000C0EB0808CAF80830002BE7D1002005B0D0
:1023A000BDE8F08F21460198FFF746F8002840F07D
:1023B0003A81A389356803F002081FFA88F00028E3
:1023C000CFD113F001095BD14F4602961FB39A0596
:1023D000D4F808802CD54745C246C0F0A48013F439
:1023E000906F40F0B18020685246494600F012FAE2
:1023F000A0682368C8EB00005344A06023603846FF
:10240000029A93681B1A81443F1A9360002BC5D02F
:10241000A389002FDBD1D5F800906F680835D5E788
:10242000D5F80090D5F8048008359FE70020704764
:1024300020682369984203D861698F4280F0B78091
:10244000B84528BFB8464246494600F0E3F9A368BC
:102450002268C8EB03034244A3602260002B49D1E9
:1024600021460198FFF7FAF8002843D0B4F90C3060
:1024700043F040034FF0FF30A38105B0BDE8F08F7B
:102480008046029082468146B9F1000F2AD0029B15
:10249000002B4CD0206823696269C845C34628BF19
:1024A000CB4698425F4604D9A36813449B4500F38A
:1024B0009080934520DB1346A76A216A0198524613
:1024C000B847071ED2DDB8EB070823D0B368DB1B83
:1024D000BA44C7EB0909B360002B3FF45FAFB9F111
:1024E000000FD4D10023D5F800A0D5F804900293B2
:1024F0000835C9E7404683E75A46514600F08AF955
:10250000A2682368CBEB02025B44B8EB0708A26029
:102510002360DBD121460198FFF7A0F80028A5D160
:10252000CDF80880D2E72068B846BA465CE74A464C
:102530000A21504600F084F800286FD001300123B2
:10254000CAEB00080293A5E762692068216902EBE3
:102550004208C1EB000A08EBD8780AF101004FEA03
:10256000680838444045424684BF804642465B0581
:1025700042D511460198FFF7D3FA8346002855D07B
:102580005246216900F0ACF8A38923F4906343F02C
:102590008003A381CAEB08030BEB0A00C4F8148084
:1025A000C4F810B02060A360B846BA461CE76FF0CC
:1025B0000043BB4228BF3B464A4693FBF1F30198D8
:1025C000A66A01FB03F3216AB04700283FF718AF62
:1025D0004CE71A465146039300F01CF92268039B0E
:1025E00001981A4422602146FFF738F8039B00281F
:1025F0007FF43CAF1F4666E7019800F06FF9834611
:102600000028C7D1019D21692846FFF743FAB4F994
:102610000C300C2223F080032A6029E7012309F102
:102620000108029336E74FF0FF30B8E6019A0C2319
:102630001360B4F90C301BE700FCFF7F00000000C2
:1026400001F0FF01102A2BDB10F0070F08D010F863
:10265000013B013A8B422DD010F0070F42B3F6D167
:10266000F0B441EA012141EA014122F007047FF080
:1026700000070023F0E80256083C85EA010586EAD7
:10268000010685FA47F5A3FA87F586FA47F6A5FA13
:1026900087F68EB9EED1F0BC01F0FF0102F007021F
:1026A00032B110F8013B013A83EA010313B1F8D1CA
:1026B0000020704701387047002D06BF35460338AB
:1026C000073815F0010F07D1013015F4807F02BFE4
:1026D000013015F4C03F0130F0BC0138704700BF35
:1026E000844641EA000313F003036DD1403A41D31D
:1026F00051F8043B40F8043B51F8043B40F8043BDC
:1027000051F8043B40F8043B51F8043B40F8043BCB
:1027100051F8043B40F8043B51F8043B40F8043BBB
:1027200051F8043B40F8043B51F8043B40F8043BAB
:1027300051F8043B40F8043B51F8043B40F8043B9B
:1027400051F8043B40F8043B51F8043B40F8043B8B
:1027500051F8043B40F8043B51F8043B40F8043B7B
:1027600051F8043B40F8043B51F8043B40F8043B6B
:10277000403ABDD2303211D351F8043B40F8043B0B
:1027800051F8043B40F8043B51F8043B40F8043B4B
:1027900051F8043B40F8043B103AEDD20C3205D31B
:1027A00051F8043B40F8043B043AF9D2043208D013
:1027B000D2071CBF11F8013B00F8013B01D30B8885
:1027C00003806046704700BF082A13D38B078DD063
:1027D00010F003038AD0C3F10403D21ADB071CBF35
:1027E00011F8013B00F8013B80D331F8023B20F89F
:1027F000023B7BE7043AD9D3013A11F8013B00F8D8
:10280000013BF9D20B7803704B7843708B7883705F
:10281000604670478842F0B50DD98B1898420AD2AD
:102820008118002A51D09A1A13F8014D01F8014D70
:102830009342F9D1F0BD0F2A48D941EA00039B0722
:1028400046D100F1100401F11003154653F8106C45
:1028500044F8106C53F80C6C44F80C6C53F8086C8A
:1028600044F8086C103D53F8046C44F8046C0F2DC8
:1028700003F1100304F11004E8D8A2F1100323F0CF
:102880000F0302F00F0E1033BEF1030F194403447F
:1028900021D91E1F0D467446043C55F8047B46F8AA
:1028A000047F032CF8D8AEF1040424F003040434AC
:1028B0002344214402F0030262B1013B0A4411F8AF
:1028C000014B03F8014F8A42F9D1F0BD0346F3E70B
:1028D0000346F2E7F0BD7246EEE700BFF9B1F8B586
:1028E00006461546B2B10C4600F01CF8854201D8E8
:1028F0002046F8BD29463046FFF712F9074668B171
:102900002A462146FFF7ECFE30462146FFF7C2F883
:102910003846F8BDFFF7BEF82846F8BDF8BD1146A9
:10292000FFF7FEB851F8040C0028BEBF091851F893
:10293000043CC018043870474E4D492048414E446D
:102940004C45520048415244204641554C54204881
:10295000414E444C4552004D454D204D414E41475E
:10296000452048414E444C45520042555320464173
:10297000554C542048414E444C4552005553414714
:1029800045204641554C542048414E444C45520048
:102990004445425547204D4F4E2048414E444C45FA
:1029A000520044554D4D592048414E444C4552002B
:1029B0002A2A2A2052494F54206B65726E656C207A
:1029C00070616E69633A0A25730A0A002A2A2A206E
:1029D0007265626F6F74696E672E2E2E0A0A006D23
:1029E00061696E28293A20546869732069732052FE
:1029F000494F5421202856657273696F6E3A2055ED
:102A00004E4B4E4F574E20286275696C6464697254
:102A10003A202F686F6D652F656C6F7065732F504E
:102A2000464531352F52494F5429290A0069646CB3
:102A300065006D61696E0000004400400000020006
:102A40000300024002000240070700260048004041
:102A500000000400090C0240080C02400707002790
:102A6000003001400700024006000240050002401D
:102A700004000240050000000010000001000000FA
:102A8000003800400F0402400E0402400D040240D2
:102A90000C0402400500000000400000000000009F
:102AA0000A5465737420666F72207065726970686D
:102AB0006572616C2054494D4552730A005468692F
:102AC0007320746573742077696C6C2074657374FB
:102AD00020616C6C20636F6E666967757265642037
:102AE0007065726970686572616C2074696D657279
:102AF00073206F66207468650A7461726765746517
:102B00006420706C6174666F726D2E20466F722047
:102B1000656163682074696D65722C206974207723
:102B2000696C6C20736574206561636820636861FB
:102B30006E6E656C20776974680A616E20696E63D9
:102B400072656D656E74696E672074696D656F7509
:102B5000742E204348302073657420746F20356DC7
:102B6000732C2043483120746F2031306D732C203A
:102B700043483220746F2031356D730A616E6420D2
:102B8000736F206F6E2E0A496E20746865206F7512
:102B90007470757420796F752073686F756C64201C
:102BA0007365652074686174206576657279206349
:102BB00068616E6E656C2066697265642C20616662
:102BC00074657220616E0A6576656E6C7920646941
:102BD00073747269627574656420616D6F756E746B
:102BE000206F662074696D65202D3E207468652015
:102BF00073686F776E20646966662076616C7565B0
:102C0000732073686F756C640A62652070726574F6
:102C10007479206D75636820657175616C20287406
:102C20006F20736F6D65206A69747465722E2E2E25
:102C3000290A54686973207465737420646F65731E
:102C400020686F7765766572204E4F542073686FE9
:102C5000772C206966207468652074696D656F75CE
:102C60007473207765726520636F72726563742078
:102C7000696E0A72656C6174696F6E20746F20747E
:102C80006865206578706563746564207265616C41
:102C90002D74696D65207E2075736520652E672E05
:102CA0002074657374732F7874696D65725F6D73CA
:102CB0006720666F720A746869732E0A0A0041768B
:102CC00061696C61626C652074696D6572733A202C
:102CD00025690A000A54657374696E672054494D6A
:102CE00045525F25753A0A0054494D45525F257596
:102CF0003A204552524F52206F6E20696E697469B6
:102D0000616C697A6174696F6E202D20736B6970D4
:102D100070696E670A0A0054494D45525F25753A3D
:102D200020696E697469616C697A6174696F6E207B
:102D30007375636365737366756C0A0054494D451A
:102D4000525F25753A2073746F707065640A005481
:102D5000494D45525F25753A20736574206368615B
:102D60006E6E656C20257520746F2025750A0054E1
:102D7000494D45525F25753A204552524F522073B6
:102D8000657474696E6720616E79206368616E6E28
:102D9000656C0A0A0054494D45525F25753A207307
:102DA00074617274696E670A0054494D45525F251B
:102DB000753A206368616E6E656C202569206669CE
:102DC00072656420617420535720636F756E7420A0
:102DD00025387500202D20696E69743A20253875D4
:102DE0000A00202D20646966663A202538750A009D
:102DF0000A544553542053554343454544454400E4
:102E00000A54455354204641494C454400000000B3
:102E100000000040FFFFFFFF01000000001C000059
:102E2000000C0040FFFFFFFF080000000032000020
:102E30000202000028020020430000000000000001
:102E40000000000000000000000000000000000082
:102E50000000000000000000000000000000000072
:102E60000000000000000000000000000000000062
:102E70000000000000000000000000000000000052
:102E80000000000000000000000000000000000042
:102E9000000000000000000000000000232D302B87
:102EA00020000000686C4C006566674546470000DE
:102EB0003031323334353637383941424344454670
:102EC0000000000030313233343536373839616232
:082ED000636465660000000068
:102ED8008C0B00200000000064030020400000006C
:102EE80000000000000000002D2A0008322A000817
:102EF8000101010128020020000000007C2E0008CA
:102F08005C2E00083C2E00080000000000000000B5
:102F18000000000000000000382E0008000000003B
:102F28000000000000000000000000000000000099
:102F38000000000000000000000000000000000089
:102F48000000000000000000000000000000000079
:0C2F58000000000000000000210000004C
:04000005080004BD2E
:00000001FF
